:100000000C9474010C949D010C949D010C949D0121
:100010000C949D010C949D010C949D010C94BD03C6
:100020000C949D010C949D010C949D010C949D01D8
:100030000C949D010C949D010C949D010C949D01C8
:100040000C949D010C949D010C948B040C949D01C7
:100050000C9448040C949D010C949D010C949D01FA
:100060000C949D010C949D01437934436F6465A009
:10007000012220B0002020F0FF00010002810200D8
:10008000FFFF003D00024B0240FFFF00010001386E
:1000900002F0FFFF000700000D02F8FFFF00010063
:1000A00001FA01FAFFFF00010001E701FCFFFF0078
:1000B0000200019F010000000E0000001F00000070
:1000C000001F1F1F1F1F1F1F1F1F1F1F1F00110AA1
:1000D000040A11001F001F101C101F001F1F111108
:1000E000111111111F00000100000000FFFF0000AE
:1000F000000001000020C8070180D0080101770836
:1001000001000000000200000200000001000000E9
:10011000010000000102720803000000020000005C
:10012000020000000220C8070140C8070104CA08F5
:100130000400000003109B08030872080000000080
:100140000400000004005EBCE2613FDD83C29C7ECF
:1001500020A3FD1F419DC3217FFCA2401E5F01E340
:10016000BD3E6082DC237D9FC1421CFEA0E1BF5DDD
:100170000380DE3C62BEE0025CDF81633D7C22C026
:100180009E1D43A1FF4618FAA427799BC584DA383F
:1001900066E5BB5907DB856739BAE406581947A5F8
:1001A000FB7826C49A653BD987045AB8E6A7F91BA1
:1001B00045C6987A24F8A6441A99C7257B3A6486DE
:1001C000D85B05E7B98CD2306EEDB3510F4E10F20B
:1001D000AC2F7193CD114FADF3702ECC92D38D6FA8
:1001E00031B2EC0E50AFF1134DCE90722C6D33D175
:1001F0008F0C52B0EE326C8ED0530DEFB1F0AE4C8E
:100200001291CF2D73CA947628ABF517490856B4CE
:10021000EA6937D58B5709EBB536688AD495CB296F
:1002200077F4AA4816E9B7550B88D6346A2B759728
:10023000C94A14F6A8742AC896154BA9F7B6E80A55
:1002400054D7896B35020403050606070708080919
:100250000901BF08010000000000000000000000CC
:100260000020000000020000020000000100000069
:100270000102000003000000020000000200000074
:100280000240000000200000008000000004BB08C5
:10029000041097080308000000000000040000009C
:1002A000042D3332373638005B437934204C696E85
:1002B00065205465737465725D00000000000000E5
:1002C000000000000000000000000000000000002E
:1002D000000000000000000000000000000000001E
:1002E000000000000003FF7C11241FBECFEFD8E008
:1002F000DEBFCDBF14BE0FB6F894A8958091600004
:10030000886180936000109260000FBE11E0A0E051
:10031000B1E0EEE4F8E202C005900D92AE36B1070E
:10032000D9F723E0AEE6B1E001C01D92AC3EB207C2
:10033000E1F70E94800D0C9425140C940000EF92BC
:10034000FF920F931F93CF93DF9300D000D0CDB7D0
:10035000DEB77C018B010E94E30C9A838983CE0176
:1003600001960E9468078B83CE0101960E946B075D
:100370008C83AE014D5F5F4FB801C7010E944A0DEB
:100380008B8189838C818A83CE0101960E947C07B0
:10039000882321F0C8010E9497070EC0CE01019664
:1003A0000E946E078823B1F389819A810E94E10C33
:1003B00089819A810E9456120F900F900F900F9092
:1003C000DF91CF911F910F91FF90EF900895CF9300
:1003D000DF93EB01CB010E94A607FC0180818E35E3
:1003E00021F4DF91CF910C94D204CE01DF91CF9113
:1003F0000C949707CF93DF93EB01CB010E94A607E4
:10040000FC0180818E3521F4DF91CF910C94CF04D3
:10041000CE01DF91CF910C949707FF920F931F931A
:10042000CF93DF93EC018B01CB010E949D07F62E49
:10043000CE010E94440DF61AD0E0CD2FCF0DC80199
:100440000E94A307D81770F4C8010E94A807EC2FD8
:10045000F0E0E159FF4FE491DC01AD0FB11DEC93E9
:10046000DF5FEBCFDF91CF911F910F91FF90089548
:10047000CF93DF93EB01CB010E94A607FC018081A3
:100480008E3521F4DF91CF910C940D12CE01DF91C6
:10049000CF910C949707EF92FF920F931F93CF93F6
:1004A000DF93CDB7DEB7ED970FB6F894DEBF0FBE82
:1004B000CDBF8C017B014DE350E0BE016F5F7F4FEC
:1004C0008AE090E00E940412AE014F5F5F4FB701D7
:1004D000C8010E944A0D1DAE4DE350E06AE070E095
:1004E000CE0101960E940612ED960FB6F894DEBF7B
:1004F0000FBECDBFDF91CF911F910F91FF90EF9075
:100500000895EF92FF920F931F93CF93DF9300D044
:10051000CDB7DEB78C017B0141E050E0BE016F5FDB
:100520007F4F87E490E00E94041289818A83AE01A4
:100530004E5F5F4FB701C8010E944A0D8A81843027
:1005400048F4898341E050E067E470E0CE01019611
:100550000E9406120F900F90DF91CF911F910F9183
:10056000FF90EF90089586E790E00E94C50C0E94EE
:1005700031120E94E10C0C94A80FCF93DF931F92CD
:10058000CDB7DEB741E050E0BE016F5F7F4F87E43B
:1005900090E00E9404120E94D6042981223031F09A
:1005A000233071F0213079F481E00EC09C01207875
:1005B000327081E02038310509F080E0817004C09C
:1005C0000E94A80501C080E00E94C8050F90DF913D
:1005D000CF910895CF92DF92EF92FF920F931F93E6
:1005E000CF93DF93CDB7DEB72B970FB6F894DEBF6E
:1005F0000FBECDBF8BE0E82E8E010F5F1F4F0E9414
:10060000760D882309F479C080916E01882301F169
:1006100081E00E94B605882359F082E091E00E94B3
:10062000D911882309F10E94D10F10926E0125C0C3
:1006300082E091E00E94F211883E934028F40E94EB
:10064000F20FFF24F39401C0F12C10926E0117C039
:1006500081E00E94AF05882349F081E080936E011C
:1006600082E091E00E949A11F12C09C080E00E9482
:10067000AF058823C9F30E94B10FFF24F3940E94B1
:10068000CE056C018091000190910101C816D90638
:1006900029F0D0920101C092000103C0FF2009F4AB
:1006A000AECFF8012E2D11922A95E9F76EE171E097
:1006B000C8010E94B31088EEC81683E0D80630F057
:1006C00063E271E0C8010E94B3100DC0E4E6CE16EB
:1006D000D10424F460E2C8010E94A51041E0B601F3
:1006E000C8010E94291166E5C8010E94A510C80131
:1006F0000E9499110E94D30582CF2B960FB6F894D1
:10070000DEBF0FBECDBFDF91CF911F910F91FF9044
:10071000EF90DF90CF900895089589E490E00197DD
:100720000000E9F70895F89498E088E10FB6F8948E
:10073000A895809360000FBE90936000E0E0F1E028
:1007400080E099E08193E030F907E0F3FFCF29984A
:1007500028988EBD0DB407FEFDCF289A0C948D030A
:1007600087FF01C078940895299A28988EBD0DB40A
:1007700007FEFDCF289A0C948D031F920F920FB69F
:100780000F9211242F938F939F93EF93FF93809158
:10079000AE029091AF0201969093AF028093AE02A9
:1007A00080918A0190918B010196883E23E0920707
:1007B00029F090938B0180938A010DC010928B01D8
:1007C00010928A018091AC029091AD0201969093B3
:1007D000AD028093AC024C9B02C080E001C082E07D
:1007E00099B195FB992790F921E09227980F809174
:1007F0008901E92FF0E024E0829FE00DF11D112432
:10080000EB51FF4FE49180918801E80FE09388015C
:1008100090938901E23031F0EE3F59F480918D01DF
:10082000815003C080918D018F5F80938D01109264
:10083000880180915D0286958695869590E0049763
:10084000ECF480915D02887F98E0980F80915D02C2
:100850008770892B80935D0280915D0286958695D5
:10086000869590E0049754F0E0919301F0E0EE0F4C
:10087000FF1FEB56FE4F808181608083FF91EF91D7
:100880009F918F912F910F900FBE0F901F901895F1
:100890001F920F920FB60F9211248F939F93EF9395
:1008A000FF9380915D0281FD07C080915D028460AD
:1008B00080935D0210925F0280915D028D7F809334
:1008C0005D028091600290915F02911106C090914B
:1008D0005D029E7F90935D0213C0E82FF0E0EF5918
:1008E000FD4F908190935E0290819093C6008F5F40
:1008F0008B3409F480E090915F02915090935F02F5
:1009000080936002FF91EF919F918F910F900FBEA6
:100910000F901F9018951F920F920FB60F921124EF
:100920008F939F93EF93FF939091C60080915D0208
:10093000877080935D0280915D0280FF09C0809185
:100940005E02981305C080915D02826080935D0213
:1009500080919301E82FF0E0EE0FFF1FEB56FE4F62
:1009600091838F5F843609F480E09091940189131C
:100970000BC0E0919301F0E0EE0FFF1FEB56FE4F2E
:1009800080818160808302C080939301FF91EF9109
:100990009F918F910F900FBE0F901F9018951092FE
:1009A0008C01089581E080938C010895CF93DF93AB
:1009B0008FB7F894C091AE02D091AF020E94B003FD
:1009C000CE01DF91CF910895CF93DF938FB7F89445
:1009D000C091AC02D091AD020E94B003CE01DF9174
:1009E000CF9108959C01CB01B9010C94F3130C94A1
:1009F0000314CF938FB7F89490915D0290FD0AC0D5
:100A000020915D0226952695269530E0C1E02430A0
:100A100031050CF4C0E00E94B0038C2F8170CF919F
:100A20000895CF93DF93C82F8FB7F894D0915F02CA
:100A30000E94B003DB34C1F38FB7F89490915D024C
:100A400092FD24C090915D0290FF12C0E09160027F
:100A500090915F02E90FEB3408F0EB54F0E0EF59AE
:100A6000FD4FC08390915F029F5F90935F020EC025
:100A700090915D02916090935D0290915D029D7FE7
:100A800090935D02C0935E02C093C600DF91CF9148
:100A90000C94B003CF938FB7F894C0915D02C170EE
:100AA0000E94B0038C2FCF910895CF938FB7F89405
:100AB000C0915D02C2FBCC27C0F990915D029B7F83
:100AC00090935D020E94B0038C2FCF910895CF9335
:100AD000DC018FB7F894C0E090919401E92FF0E029
:100AE000EE0FFF1FEB56FE4F208120FD0EC0209120
:100AF0009301921751F0319620812C939F5F943689
:100B000009F490E090939401C1E00E94B0038C2F0F
:100B1000CF910895CF938FB7F89490919401E92FD6
:100B2000F0E0EE0FFF1FEB56FE4FC081C170209129
:100B30009301921719F090819E7F90830E94B003D9
:100B400081E08C27CF91089589E1809392010895E7
:100B500081E090919201911101C080E00895E82F09
:100B6000F0E0E057FE4F808110820895E82FF0E01A
:100B7000E257FE4F80810895CF938FB7F894C091CC
:100B80008D0110928D010E94B0038C2FCF9108959A
:100B9000882311F05E9A08955E98089580910E0161
:100BA00090910F0108950F931F93CF93DF938C01C2
:100BB000F801C1918F01CC2391F1CA3071F0CD3091
:100BC000C1F482E00E94A70310928701C2E3D0E043
:100BD0000E948D032197E1F7EBCF81E00E94A703EC
:100BE00010928701C2E3D0E00E948D032197E1F7C4
:100BF000DFCF80EF8C0F883008F4C82FD0918701A9
:100C0000D11104C080E80E94A70302C0D83080F64A
:100C10008C2F0E94B403DF5FD0938701C9CFDF918F
:100C2000CF911F910F9108950F931F93CF938091B0
:100C30008C0181110E949303F8949FE088E10FB624
:100C4000F894A895809360000FBE909360008FE3A6
:100C500084B981E085B98DE387B918B880EC8AB989
:100C60008CE38BB90E948D0387E880937A00809192
:100C70007A00806480937A0082E08093B00083E001
:100C80008093B10082E78093B3008091700082600E
:100C9000809370008BE090E09093C5008093C40037
:100CA0001092C00088ED8093C10086E08093C2005E
:100CB0008DE58CBD2A9A04EF11E00E948D0301504E
:100CC0001109D9F780E30E94A70380E30E94A703DC
:100CD00081E30E94A70384E10E94A70384E70E94A6
:100CE000A70381E50E94A7038AE60E94A70304ECFC
:100CF00019E00E948D0301501109D9F78CE00E9480
:100D0000A70386E00E94A70380E30E94A70305EBE8
:100D100010E0C0E48C2F0E94A703F80184910E9488
:100D2000B403CF5F0F5F1F4FC037A1F7789482E005
:100D300080938C01CF911F910F91089581E0909144
:100D40008C01923009F080E00895CF93DF93A8954D
:100D50008AE091E00E94E111882309F448C081E40F
:100D600080937C0080917A00806480937A008091E7
:100D70007A0086FDFCCFA091780080917900B0E0E8
:100D8000B82BA11584E0B80720F4A11580E8B807B6
:100D900039F480E090E890930F0180930E0117C022
:100DA00024EE3CE00E94B21326EF37E240E050E030
:100DB0000E949313285F3F4F37FD05C030930F010A
:100DC00020930E0104C010920F0110920E01609149
:100DD0000E0170910F0186E091E00E94181086E0EC
:100DE00091E00E94301090930F0180930E010E94B9
:100DF000D6042091720130E0AC0155272417350745
:100E000059F40E94D60420916F0130E0AC015527BF
:100E100024173507C1F540C080937201E0E7F1E087
:100E2000AEE8B1E0C0E9D1E090E031E04AE052E361
:100E300089B1913029F082FB882780F9832705C08A
:100E4000869586958695892781702C91222339F085
:100E5000811103C02081211107C0508309C088235C
:100E600031F02081222319F02150208301C04083DA
:100E70002191211102C08C9388839F5F1196219646
:100E80009230B1F6BECF80936F018091920188239A
:100E900019F0815080939201DF91CF9108950E94C3
:100EA0004A058111FCCF80918C01882361F081304B
:100EB00061F4E0E0F8E7859194918C30944929F44D
:100EC0000C94023C08950E9493030895962F089570
:100ED000FC0180810895FC0181810895FC018081DD
:100EE0008F3F39F491E081818F3F09F490E0892FA1
:100EF00001C081E081700895FC018081882331F078
:100F000091E08181811190E0892F01C081E08170A1
:100F100008950F93FC0181E08083118273836283C3
:100F2000248335834683578300870F910895FC01FE
:100F300010820895FC0180810895FC01648175810F
:100F4000868197810895FC0180850895099608950A
:100F500009960895DC019BE4E5E5F3E001900D922C
:100F60009A95E1F7109254030895E3EBF2E0818142
:100F700080958370806C8183828184838381858363
:100F8000A2E1B1E08C91828311968C9183830895C4
:100F90000E94B5071092B3020895EF92FF920F934B
:100FA0001F93CF93DF93DC012C9130E08901E4E0C3
:100FB000000F111FEA95E1F7A0E0B0E0C0E0D0E03B
:100FC000F801EA0FFB1FE40FF51FF490FF2061F119
:100FD000FB01E080EF2DEE2111F1220F331F220FD4
:100FE000331F2C0F3D1F220F331F220F331FF90118
:100FF0003196E40FF51F65917491F9013396E40F72
:10100000F51FE491DC01EC936115710569F0FB01BA
:10101000DF91CF911F910F91FF90EF90099421964E
:101020001496A031B10561F6DF91CF911F910F9118
:10103000FF90EF900895FC01DB0181E090819A3AE6
:1010400009F080E08C938181815C91E0823008F42A
:1010500090E011969C931197848112968C9312972D
:10106000858113968C931397468150E060E070E081
:10107000BA01552744278085480F511D611D711DF8
:10108000878190E0982F8827480F591F611D711D97
:1010900014964D935D936D937C9317979185189655
:1010A0009C931897818180FF09C03A96199680E039
:1010B000891721F021912D938F5FFACF08951F9307
:1010C000CF93DF93EC01162F0E94D604810F911D60
:1010D000009711F481E090E099838883DF91CF91AC
:1010E0001F9108956AEF80E093E00C945F0883EB12
:1010F00092E00E94AA0762E38EEF92E00C945F08F0
:10110000CF93DF93EC010E94D60483709927019658
:1011100090911001890F803108F083E080931001D5
:1011200060911001CE01DF91CF910C945F088EE4A5
:1011300093E00C9480088EEF92E00C9480080F935B
:101140001F93CF93DF93FC01218120FF03C0118502
:10115000155F01C01BE0082FC82FD92F8C2F801BD3
:10116000811720F489910E941105F8CFDF91CF916A
:101170001F910F91089583E093E00C949F0883E002
:1011800093E00E94AA076AEF80E593E00E945F085F
:101190000C94A40583EB92E00E949F080C94A40594
:1011A0000E94B50762E38EEF92E00C945F08CF9245
:1011B000DF92EF92FF920F931F93CF93DF93EC0197
:1011C0008B017A016901809154038823B1F18091E8
:1011D000560381FF06C080915203816080935203C1
:1011E0002CC090911101943041F1911124C0817073
:1011F00091E089272091B402217092278917D9F0B4
:1012000085E492E0FC01A4913196E491B0E0AB5A00
:10121000BC4FF0E0ED54FD4F3C91208132130BC0E8
:101220000296F2E081359F0769F7809102038160A1
:101230008093020302C010925403809153038430C0
:10124000E1F0809111018430C1F00E94F9048823FB
:10125000A1F0F70180819181892B61F00E94D60471
:10126000F70120813181281B390B121613062CF04F
:1012700011821082888184608883F8018081918145
:10128000892B61F00E94D604F80120813181281B4E
:10129000390B121613062CF011821082888180629D
:1012A0008883F3E0C235DF07A1F4809153038430D3
:1012B00009F50E944A0581111DC00E9455059091B3
:1012C0005203882311F0906101C0986090935203FB
:1012D00011C080911101843069F40E944A05811186
:1012E00009C00E9455059881882311F0906101C0C2
:1012F00098609883F6018281882331F081E09381A0
:10130000992319F080E001C081E080FF03C088814B
:1013100080688883F60180818A3A19F08881806428
:101320008883DF91CF911F910F91FF90EF90DF9015
:10133000CF90089523E033E04EE453E060E573E09E
:1013400082E593E00E94D70841E552E062E573E050
:1013500083E593E00E94CD0710925203089523EB9A
:1013600032E04EEF52E060E073E082E093E00E94F2
:10137000D70845EF50E062E073E081E191E00E9420
:10138000CD07109202030895DF92EF92FF920F9320
:101390001F93CF93DF93FB011082FC012081222356
:1013A00009F48CC0FF24F3942181213009F4F12C3D
:1013B000F2E0633B7F0709F4F094EB018C01FC0140
:1013C00032812381635B724091F0DC80D31276C05E
:1013D000ED80E21273C08A8191E0882319F02B819D
:1013E000211190E090FF64C0E12CD12C61C080916C
:1013F0001201909113014AEA48834F2D4370406CCB
:1014000049833A832B838C839D83F80186818E8365
:1014100085818F83848188878085813410F48987D2
:1014200001C01986DE01CE010A96EFEF2D91E22769
:10143000F0E0EB5BFE4FE491A817B907B9F7F0FEB7
:1014400019C080E09985891798F4282F30E0D801D9
:10145000A20FB31F19969C91DE01A20FB31F1A961B
:101460009C93E927F0E0EB5BFE4FE4918F5FEACFBE
:10147000865F01C08AE0DE01A80FB11DEC938A816E
:10148000882331F081E09B81992319F080E001C02D
:1014900081E080FF13C08981833C29F49E81907F85
:1014A00081E0903E09F080E080FD08C0188206C00F
:1014B0006B810E9466073D2D2E2D9DCFDF91CF9130
:1014C0001F910F91FF90EF90DF900895909313017B
:1014D0008093120108958091120190911301089553
:1014E000CF93DF93EC010E949707809153038130E3
:1014F00071F4BE0183E093E00E941B0880915203C7
:101500008260809352030E949A0981E001C080E0CA
:10151000DF91CF91089520915303223069F463E065
:1015200073E00E94C4098091520382608093520349
:101530000E949A0981E0089580E0089520911101A8
:10154000223069F463EB72E00E94C40980910203C7
:101550008260809302030E94AF0981E0089580E0D9
:101560000895CF93DF93EC010E94970780911101BA
:10157000813071F4BE0183EB92E00E941B088091E0
:1015800002038260809302030E94AF0981E001C0E0
:1015900080E0DF91CF91089581E090911101923028
:1015A00009F080E008951092530382E080931101C6
:1015B00010925403E2E1F1E08FEF8083818308957C
:1015C0000F931F93CF93DF931F92CDB7DEB7809118
:1015D0005403811181C00E948A05811102C01092BA
:1015E000B2021AE00FEFCE0101960E946705882330
:1015F00009F472C09091B202E981913059F018F06B
:10160000993081F01CC0EA3A71F71093B10200934F
:10161000B00215C08E2F86958695803381F010928A
:10162000B202E1CF8FEF8E0F8034C8F7809156035E
:1016300080FF05C08091B1028E0F8093B102A92F67
:10164000B0E0AB5ABC4FEC938091B002E827F0E0D9
:10165000EB5BFE4FE491E093B0028091B1029813EE
:1016600037C01092B202E11137C0809157039091B8
:101670001201891711F081112FC090915803209108
:101680001301921711F0911127C0209159032223C1
:1016900019F120915A032223F9F0882329F081E0DF
:1016A000992319F080E001C081E080FF0DC0809196
:1016B0005603833C31F490915B03907F81E0903E30
:1016C00009F080E080FF08C081E08093540304C0EB
:1016D0009F5F9093B20287CF0E949A090E94AF0940
:1016E0000F90DF91CF911F910F9108958091530337
:1016F0008350823018F40E949A09F8CF089580919F
:10170000DC03882369F09091DD039F5F9F3019F01F
:101710009093DD0302C01092DD0381508093DC03BF
:1017200008958F929F92AF92BF92CF92DF92EF92E5
:10173000FF920F931F93CF93DF93CDB7DEB7299717
:101740000FB6F894DEBF0FBECDBF8C012091DE0333
:10175000211104C0C8010E9497077EC0FC01C4800B
:10176000D580E680F7806091DF037091E003FB0194
:1017700085919591A591B491C816D906EA06FB0604
:1017800048F3215030E0822F022E000C990B831B6E
:10179000910937FD939597FD019695958795830F50
:1017A000FB0199E08902E00DF11D112485909590CF
:1017B000A590B4908C149D04AE04BF0418F431E0DD
:1017C000380F07C0C814D904EA04FB0438F42FEF1B
:1017D000280F231724F08213D6CF01C0282FE9E069
:1017E0002E02600D711D112449E050E0CE010196DA
:1017F0000E94EA13F80191818F81911103C0813019
:1018000039F4A8CF913009F0A5CF882309F4A2CFED
:101810002D813E8189819A81AB81BC81820F931F8A
:10182000A11DB11DF8012085C20ED11CE11CF11CC7
:101830008C159D05AE05BF0508F48CCFE885F985AC
:10184000309709F487CFB801CE0101960995F801C8
:101850008081882309F47ECF29960FB6F894DEBFE5
:101860000FBECDBFDF91CF911F910F91FF90EF90F1
:10187000DF90CF90BF90AF909F908F900895CF92C0
:10188000DF92EF92FF920F931F93CF93DF93CDB729
:10189000DEB7C954D1090FB6F894DEBF0FBECDBF75
:1018A0008091DC03882309F460C0E090DD0384E0CC
:1018B000E89E70011124D701A056BC4F6D018D9197
:1018C0009C91892BF1F10E94CC0A882309F44DC028
:1018D0008E010F5F1F4F89E4F80111928A95E9F795
:1018E000D601ED91FC91C8010995C8010E949A07A3
:1018F000882321F1F60111821082DB800E946B0A9D
:10190000D81218C0DC800E946B0AD91213C08981DA
:10191000882319F0C8010E94910BF701E056FC4F93
:10192000E280F3800E947F0BE114F104F1F0C80122
:10193000F7011AC0C8010E949E0A17C00E947F0BBF
:1019400014C0CE0101960E94B10A882371F0D6011D
:1019500012960D911C9113970E947F0B0115110592
:1019600021F0CE010196F8010995C75BDF4F0FB654
:10197000F894DEBF0FBECDBFDF91CF911F910F91C5
:10198000FF90EF90DF90CF9008959C0190E021159B
:10199000310581F0F90189E0989FE00DF11D1124D6
:1019A00045915591659174919F5F4C3F5F4F6F4F8B
:1019B000710581F73093E0032093DF039093DE03FA
:1019C00008950C94660A0E946B0A08959C019091F8
:1019D000DC039F30A9F0E091DD03E90FEF3008F060
:1019E000EF5084E0E89FF0011124E056FC4F318372
:1019F0002083738362839F5F9093DC0381E008956B
:101A000080E008950E94D30A1092E0031092DF0351
:101A10001092DE031092DD031092DC030895CF9341
:101A2000DF93CDB7DEB7C954D1090FB6F894DEBF46
:101A30000FBECDBF0E94E00ACE0101960E94700A3F
:101A4000882359F08981882321F0CE0101960E94D4
:101A5000910BCE0101960E948B0A0E943F0CC75B3E
:101A6000DF4F0FB6F894DEBF0FBECDBFDF91CF9131
:101A700008950E94CC0A811105C00E943F0C0E946B
:101A8000E00AF7CF0C94760BFC01608171818281B2
:101A900093810895DC01FB0194818C91981B892F1F
:101AA0009181992321F0913001F590E00EC0DB0186
:101AB00019969085980F891739F0FA01E80FF11DF2
:101AC00020812D938F5FF7CF0895392F380F208510
:101AD000921758F4DF01A90FB11D19962C91DA0164
:101AE000A30FB11D2C939F5FF0CF08950E94A50610
:101AF0000E94D7120E940F0D0E94BD020C949E06F8
:101B00000E9414060E947F120E94020D0E94B302DE
:101B10000E94EA020E948C030E94390D0E947513F4
:101B20000C944F07CF93DF9300D000D0CDB7DEB732
:101B300028EE33E0482F429FC001439F900D1124AF
:101B400089839F738A818078892B80688A831C822D
:101B50001B82CE0101960E949A11CE0101960E942D
:101B6000D911811104C00E94760D8111F6CF0F901A
:101B70000F900F900F90DF91CF91089580E00E9419
:101B8000AF0581E00E94AF050C94BC050F931F9335
:101B9000CF93DF938C01C1EED3E0E991E43028F4D8
:101BA000F0E0ED59FE4F608101C06FE3C8010E9473
:101BB000A51083E0C93ED80781F7DF91CF911F912F
:101BC0000F9108950F931F93CF93DF93CDB7DEB797
:101BD0002B970FB6F894DEBF0FBECDBF0E949A07B9
:101BE000E091E903F0E0EF51FC4F882311F082E02F
:101BF00001C083E080838E010F5F1F4F8BE0F801EF
:101C000011928A95E9F76DE0C8010E94A510C801FC
:101C10000E94C60DC8010E9499110E94D3058091AF
:101C2000E9038F5F8093E9032B960FB6F894DEBF2C
:101C30000FBECDBFDF91CF911F910F910895EF920D
:101C4000FF920F931F93CF93DF93CDB7DEB72D97FE
:101C50000FB6F894DEBF0FBECDBF7C0142E050E06E
:101C6000BE01645F7F4F88E490E00E9404126C859F
:101C70007D8507E020EF3FEF4FEF50E0C7010E9466
:101C80008907E091E903F0E0EF51FC4F81E08083A8
:101C90008E010F5F1F4F8BE0F80111928A95E9F7D3
:101CA0006DE0C8010E94A510C8010E94C60DC801C0
:101CB0000E9499110E94D3052D960FB6F894DEBFAD
:101CC0000FBECDBFDF91CF911F910F91FF90EF908D
:101CD00008950F931F93CF938C01C62F643648F459
:101CE00060E30E94A510CA3020F460E3C8010E949E
:101CF000A5106C2F70E0C801CF911F910F910C942B
:101D0000D9107F928F929F92AF92BF92CF92DF9223
:101D1000EF92FF920F931F93CF93DF93CDB7DEB770
:101D200065970FB6F894DEBF0FBECDBF5C010E9471
:101D3000BE0DF501808191819D8B8C8B8091160168
:101D400090911701A0911801B0911901888B998B7E
:101D5000AA8BBB8B80911A0190911B01A0911C0151
:101D6000B0911D018C879D87AE87BF87CE014096BD
:101D70000E949A1111E08FE7982EDD24D394C12C94
:101D8000882483949BE0792ECE0101967C01CE01BC
:101D900040960E94D911811199C00E94760D882326
:101DA00009F494C00E94BC05082F9816B1F1CE0129
:101DB00044960E946807182FCE0144960E946B0734
:101DC000682FC11002C0100F01C0600F112321F055
:101DD000662309F4B5C00EC011E010160CF4B5C0AE
:101DE000011101C010E01195611104C00111A3C0DF
:101DF00060E009C01F3F39F46F3F29F410160CF45E
:101E0000A2C001116EEF812F0E9466079D8B8C8B03
:101E1000CE0140960E949A1111E0CE010C960E94CC
:101E2000E111882311F0D82403C0112309F441C023
:101E3000F701872D11928A95E9F76DE0C7010E949D
:101E4000A510C11019C0D11002C060E201C06EE738
:101E5000C7010E94A5106C89C7010E94690ED110AC
:101E600002C06EE201C06FE7C7010E94A5106D8934
:101E7000C7010E94690E18C06C89C7010E94690ED3
:101E8000D11002C06EE201C06EE7C7010E94A5102A
:101E90006D89C7010E94690ED11002C060E201C0C5
:101EA0006FE7C7010E94A510C7010E9499110E9407
:101EB000D30581E00E94AF05882329F091E0C9167F
:101EC00029F0CC24C39410E0902E61CFCE0140962F
:101ED0000E94D911882369F0C11003C088E291E003
:101EE00002C082E391E00E94D30581E00E94920D3E
:101EF0000CC08CE391E00E94D30581E00E94920D1A
:101F00008C899D89F501918380830E94BE0D659621
:101F10000FB6F894DEBF0FBECDBFDF91CF911F91FA
:101F20000F91FF90EF90DF90CF90BF90AF909F9078
:101F30008F907F9008951F3F09F464CF6FEF63CFB8
:101F400010160CF053CF61E05ECF61115CCFFBCF78
:101F500086E491E00E94D30582E00E94920D0C94E9
:101F6000BE0DCF93DF931092E903C1EED3E0199237
:101F700062EE7DE08FE19EE00E94E60C83E0C93EC8
:101F8000D807A9F78091E903883020F40E94760DE4
:101F90008111F8CF82E00E94920DDF91CF910C94D5
:101FA000BE0DCF93DF9300D0CDB7DEB78FE491E0C5
:101FB0000E94D30581E00E94920D0E9431129A8303
:101FC0008983CE0101960E94810E89819A810E94A7
:101FD000561289819A810E94E10C0F900F90DF9137
:101FE000CF910895CF93DF9300D0CDB7DEB789E5C9
:101FF00091E00E94D30581E00E94920D42E050E002
:10200000BE016F5F7F4F88E490E00E940412CE0112
:1020100001960E94810E42E050E068E470E0CE013B
:1020200001960E9406120F900F90DF91CF910895B4
:10203000DC019C91911103C013969C9113979150D0
:1020400011962C91119712968C911297E22FF82FDE
:10205000E90FF11DE90FF11D718360839C930895D1
:102060008F929F92AF92BF92CF92DF92EF92FF92A8
:102070000F931F93CF93DF93CDB7DEB77C016DB77E
:102080007EB7DC0113968C91EDB7FEB722E0829FFC
:10209000E019F10911240FB6F894FEBF0FBEEDBF91
:1020A000ADB7BEB711964D01AD0190E0981781F123
:1020B000D7011196ED91FC9112979A0128193909CF
:1020C000DF01A20FB31F2D913C912115B0E83B0712
:1020D00041F1FA0121933193AF01292F2223B1F06D
:1020E000D401A20FB11DA20FB11DFD01B290A290AB
:1020F0008F01CD90DC901197CA14DB043CF4F801F9
:10210000D182C082AD92BC922150E8CF9F5FCECFEA
:102110009695F401E90FF11DE90FF11D8081918180
:1021200002C080E090E80FB6F8947EBF0FBE6DBF8E
:10213000DF91CF911F910F91FF90EF90DF90CF90A3
:10214000BF90AF909F908F900895FC012285293019
:1021500048F4E20FF11D60832F5FFC012287E20F3C
:10216000F11D108208950F931F93CF93DF938C017D
:10217000EB016991662321F0C8010E94A510F9CFF7
:10218000DF91CF911F910F9108950F931F93CF93DC
:10219000DF938C01EB01FE016491662329F0C801F5
:1021A0000E94A5102196F7CFDF91CF911F910F913B
:1021B0000895CF92DF92EF92FF920F931F93CF93E8
:1021C000DF937C018B0177FF17C06DE20E94A510A1
:1021D000011580E8180769F467E671E0C701DF912F
:1021E000CF911F910F91FF90EF90DF90CF900C94C3
:1021F000B310119501951109C0E1D7E220E08AE002
:10220000C82ED12CC801BE010E947F13CB01B6019C
:102210000E947F13211102C0009731F060E3680F24
:10222000C7010E94A51021E0CE01B6010E947F13D4
:10223000EB016130710511F421E0E4CF209711F733
:10224000DF91CF911F910F91FF90EF90DF90CF9092
:102250000895FF920F931F93CF93DF93EC018B01AF
:10226000F42E611580E8780731F461EA72E0CE015E
:102270000E94C5103AC077FF07C06DE2CE010E94F0
:10228000A51011950195110982E0F816E1F08F155E
:1022900020F081E0F816F1F024C083E0F81659F040
:1022A00084E0F8121EC0003187E21807D4F460E31E
:1022B000CE010E94A510083E83E0180794F460E365
:1022C000CE010E94A510043611055CF460E3CE0136
:1022D0000E94A5100A30110524F460E3CE010E948B
:1022E000A510B801CE010E94D910FF20E1F06EE2E6
:1022F000CE010E94A5102A854FEF420F30E02F1922
:102300003109842F90E0821793076CF0DE01A80F4B
:10231000B91F5C910197FE01E80FF91F80818C9332
:1023200050834150EECFDF91CF911F910F91FF90DD
:1023300008950895CF93DF93EC0188812981922F2E
:102340009F7321E0892B09F020E0898120FB87F928
:10235000898386FD03C00E94D60402C00E94E40463
:102360009B838A83DF91CF910895CF93DF93EC0114
:10237000998197FD19C096FD03C00E94D60402C042
:102380000E94E4042A813B81AC01421B530B28814B
:102390008981382F3F734217530720F4C901841BEA
:1023A000950B04C08068898380E090E0DF91CF9135
:1023B00008950E94B51121E0892B09F020E0822FB9
:1023C00008950F931F93CF938C010E94D911C82FAA
:1023D000882319F0C8010E949A118C2FCF911F9168
:1023E0000F910895CF93DF93FC01F081CF2FFC0173
:1023F0002181D22FDF730E94B5119E01281B390B5A
:10240000C901DF91CF9108950C94F2040E94F70462
:10241000109215011092140108950F931F93CF93FA
:10242000DF931F92CDB7DEB70AE010E0F801E25665
:10243000FD4FE491E98341E050E0B801CE010196FF
:102440000E94F7040F5F1F4F0A34110579F71092AD
:102450001501109214010F90DF91CF911F910F91F0
:102460000895CF93DF9300D000D0CDB7DEB744E01E
:1024700050E0BE016F5F7F4F82E090E00E94F20467
:102480008B8180959981891308C06C8160959A81B0
:10249000691303C00E94660702C098E78FEF0F9090
:1024A0000F900F900F90DF91CF910895CF93DF930E
:1024B00000D000D000D0CDB7DEB79E838D83CE0193
:1024C00005960E9468078983CE0105960E946B07D6
:1024D0008A83998190959B8380958C8344E050E01A
:1024E00062E070E0CE0101960E94F70426960FB6D6
:1024F000F894DEBF0FBECDBFDF91CF910895EF926C
:10250000FF920F931F93CF93DF9300D0CDB7DEB729
:102510002AE0E22EF12C0FEF1FEF41E050E0BE0168
:102520006F5F7F4FC7010E94F2048981082788E00E
:10253000A8015695479598012170332700FF02C0E6
:1025400028E034E88A0102271327815089F72FEF0A
:10255000E21AF20A8AE4E816F104F9F60F3F2FEFC7
:10256000120711F400E010E042E050E0BE016F5F9E
:102570007F4FC7010E94F20489819A8126E5E21605
:10258000F10439F022E0E20EF11C8F3F2FEF9207A9
:1025900059F38017910711F00E940D120F900F90C0
:1025A000DF91CF911F910F91FF90EF900895EF92DF
:1025B000FF921F93CF93DF9300D000D01F92CDB72F
:1025C000DEB780911401909115018F3F2FEF920794
:1025D00009F480C041E050E0BE016B5F7F4F0A9676
:1025E0000E94F2042091140130911501211531054A
:1025F00031F48FEF9FEF9093EB038093EA034D81CB
:102600008091EA039091EB03842748E0FC01F69562
:10261000E795BC016170772780FF02C068E074E82D
:10262000CF0186279727415089F79093EB0380933A
:10263000EA032F5F3F4F2034310529F03093150115
:102640002093140147C02FEF3FEF309315012093E3
:1026500014018F3F2FEF920719F09C838B8302C0E8
:102660001C821B8210E09AE4E92EF12C42E050E03B
:10267000BE016F5F7F4FC7010E94F20489819A817A
:102680008F3F2FEF920731F422E0E20EF11C1F5F23
:10269000173061F72B813C8182179307D9F08FEFB8
:1026A0009FEF9A83898342E050E0B701CE01019603
:1026B0000E94F7041F5F173008F010E0612F70E0F0
:1026C0006B5D7F4F660F771F42E050E0CE010396AF
:1026D0000E94F7040F900F900F900F900F90DF91D2
:1026E000CF911F91FF90EF900895809114019091E8
:1026F0001501019619F00E94D712F7CF0895AA1B71
:10270000BB1B51E107C0AA1FBB1FA617B70710F0DC
:10271000A61BB70B881F991F5A95A9F7809590950E
:10272000BC01CD010895052E97FB1EF400940E9474
:10273000AA1357FD07D00E94B91307FC03D04EF42B
:102740000C94AA1350954095309521953F4F4F4FCB
:102750005F4F089590958095709561957F4F8F4F4D
:102760009F4F08950E94DB13B7FF0895821B930BC0
:102770000895A1E21A2EAA1BBB1BFD010DC0AA1FC2
:10278000BB1FEE1FFF1FA217B307E407F50720F0DA
:10279000A21BB30BE40BF50B661F771F881F991F55
:1027A0001A9469F760957095809590959B01AC019E
:1027B000BD01CF010895A29FB001B39FC001A39FA7
:1027C000700D811D1124911DB29F700D811D11246A
:1027D000911D0895FB01DC0102C005900D9241504E
:1027E0005040D8F70895DC01CB01FC01F999FECFE8
:1027F00006C0F2BDE1BDF89A319600B40D92415089
:102800005040B8F70895DC01A40FB51F4150504067
:1028100048F0CB01840F951F2E910E941414415053
:102820005040D0F70895262FF999FECF92BD81BD73
:10283000F89A019700B4021639F01FBA20BD0FB6FE
:0E284000F894FA9AF99A0FBE0895F894FFCF13
:10284E000080B88B00000073010A658000000080D4
:10285E000302FFFFFFFF10A700002C8100000D55A3
:10286E003A200020782E78000D207878782E78780F
:10287E0078000D7878782E78787820000D2020203A
:10288E004F6B202020000A204379342D4C54000D2C
:10289E004F776E204164723A000D446573742E4179
:0E28AE006472001011121333323736380000F6
:00000001FF
